:1000000011C029C028C027C026C025C024C023C0D5
:1000100022C021C07E8D9CABB9B2A0AB3C9C1E8D92
:100020000500020011241FBECFE9CDBF10E0A0E6FD
:10003000B0E0EEEEF3E002C005900D92A237B107FA
:10004000D9F710E0A2E7B0E001C01D92A439B107D2
:10005000E1F775D0CAC1D4CF2AE733E003C0F90174
:100060003197F1F70197D8F7089590917300892F90
:100070008F5F8F71809373008EBB809172008DBBF8
:1000800084E28CBB86E28CBBE199FECF9EBB84E10F
:100090008CBB86E18CBB089540E250E060E070E0EC
:1000A00084E790E093D18091730001C08F5FE82FC7
:1000B000F0E0EC58FF4F90819F3F19F48032B0F38D
:1000C00007C080937300803218F4909372000895F3
:1000D000109273000895809172008F5F8093720078
:1000E000809172008F3010F010927200089580910C
:1000F0007200803440F480917200882321F0809156
:100100007200815009C0809172008F73833038F47F
:100110008091720080648F5F8093720008951092C6
:1001200072000895A29A81E687B986EC86B908958F
:1001300037980895369A3699FECF85B1089582E0B2
:1001400087BB81E28FBD89E083BF8FEF86BFA4DFCD
:10015000A39A83E687B986EC86B93699FECF369A9C
:100160003699FECF85B18F3B10F0B5DF07C085B162
:10017000853610F0BCDF02C01092720076DFD8DF47
:10018000BB9AC39ACFDF479A8091720086FF09C05D
:10019000E0917200EF73F0E0E15AFF4F80818093AD
:1001A0007200C8DF10E0C0E0D0E043E2F42E58E077
:1001B000E52E0FEF6CE3D62E72E0C72E8091720011
:1001C000863008F041C0FFBCE0917200F0E0ED59CC
:1001D000FF4F808189BD8091720081111AC0AADF12
:1001E00020E030E0F901E75EFF4FE491E81760F4AA
:1001F00086B7F901E65EFF4F2491821710F48F5FF6
:1002000001C0815086BF05C02E5F3F4F2A303105A7
:1002100049F785E090E020DFCF3F8FEFD80709F066
:10022000219680917200843008F497C0C13A9FE013
:10023000D90708F492C080917200815080937200B7
:1002400014DFC0E0D0E089C0809172008930E0F412
:10025000FFBC34E0B32EE0917200F0E0E15AFF4FB2
:10026000808189BD85E090E0F7DEE0917200F0E0EA
:10027000ED59FF4F808189BD81E490E0EDDEBA94B5
:1002800051F780ED92E068C0809172008A3080F46E
:1002900009BD81E090E0E0DE19BC89EF90E0DCDE92
:1002A00009BD81E090E0D8DE19BC8DEE92E054C02B
:1002B000809172008D30A8F409BD20E931E0C901B8
:1002C0000197F1F719BCE0917200F0E0ED59FF4F92
:1002D000808190E0009709F03FC0C9010197F1F7D4
:1002E0003CC0809172008D30B9F4B12C09BD81E021
:1002F00090E0B2DE19BC8DE18B1518F48D2D8B19B1
:1003000001C08B2D90E04496880F991FA5DEB39411
:100310009CE3B912EBCF21C0809172008F30E8F4DA
:1003200009DFE4E1F0E0B12C9491981708F4B3945C
:10033000319690E0E931F907B9F7A12C09C0E9BC81
:1003400084E690E089DE19BC80E991E085DEA39423
:10035000AB10F5CF80ED97E07FDE349B2FCF25B13A
:1003600030E080917200823018F483E790E002C0A0
:100370008DE790E02817390734F51F5F133020F11F
:1003800080917200863018F0C092720018C080917F
:100390007200823030F08091720081508093720040
:1003A0000EC01092720019BC85B7877E806185BF30
:1003B00085B7806285BF889585B78F7D85BF55DEFF
:1003C00080ED97E049DE10E0369AF8CEA82F862F10
:1003D000E82FE199FECF1FBA05C0EEBBE09AE39586
:0E03E0000DB20D924150C8F70895F894FFCF6A
:1003EE00050B0E0001082A78FF000108FF4F290FA8
:0203FE00FF08F6
:00000001FF
